:072E720001020310203040B3
:042E5F00C112C115C6
:102DD10075A4CDE4F5F275F3F075A6E075E106751D
:032DE100E24022AB
:102DE40075BC4475E88075BA1F75D108E4F5BB431A
:032DF400E60822CC
:0C2E3C0075A14075F809E4F5A2D2AE22A1
:091A0800E4F5B1F5A975B28322E1
:0D2E08007592027593FE75910443E68022D9
:0B2E540075CA8F75CBFFD2CAD2AD2229
:102D4D00E4F5D9121A08122DD1122DE4122E3C12CF
:082D5D002E54122E080228C9B1
:102D1A00E4FEEF30E004C2878002D287C286D28600
:092D2A00EFC313FF0EEEB402E941
:012D3300227D
:061A1B00EF04FF022D1A8A
:102DBD00AF48121A1BAF47121A1BAF46121A1BAFA0
:042DCD0045021A1B86
:02251800A90711
:10251A00E9744929F8E6FF741829F8E62FFBE43331
:10252A00FAD3EB94FFEA940040047A007BFF741418
:10253A0029F8E6FD7C00AF03AE021215B0AA06AB7D
:10254A0007EB7807CEC313CE13D8F9FB743429F8F6
:10255A00E6FD7C00AF031215B0AA06AB07EB7806BE
:10256A00CEC313CE13D8F9FBAA06C2ADE925E024DF
:09257A0029F8A60208A603D2AD5F
:012583002235
:10199400E4FF75BB11FE75E89030EDFD742B2EF558
:1019A40082E43402F583E5BEF00E05BBEEC3940277
:1019B40040E490022BE0FED394194021A3E0FDD330
:1019C40094194019EE94E85004C20A8002D20AED38
:1019D400C394E85004C2098008D2098004C209C231
:1019E4000AA20AE43325E0FFA209E4334F14600B92
:1019F40014600B14600B24037F48227F49227F4A22
:041A0400227F4B22D0
:0D2E150075347F75357F75367F75377F22E8
:101A3000122D4DE4FC12199490025EEFF00CECB400
:101A40000AF3122DE4122E15122D34122912E5B0CC
:101A5000541EF53830A403433801122E22750807AE
:0D1A60007509D0C213D2AF43E601122DBDAF
:101A6D0090022AE0FF605330E30EE518C394035053
:101A7D000775347FEF5407F090022AE0FF30E20E35
:101A8D00E519C39403500775357FEF540BF09002A1
:101A9D002AE0FF30E10EE51AC39403500775367F37
:101AAD00EF540DF090022AE0FF30E00EE51BC394D9
:101ABD0003500775377FEF540EF0E5256073146002
:101ACD004324FD601824FC602024F86028240E7047
:101ADD005A0545E545B40303E4F54580220546E581
:101AED0046B40303E4F54680160547E547B4030302
:101AFD00E4F547800A0548E548B40303E4F54812C8
:101B0D0029348027301218122E15A213B3921330D8
:101B1D001306C219C2A58013D2A5122E22800CE481
:101B2D0090026CF0122E80C215D2A5122DBDE4F5D7
:101B3D0025301144C211E50945086008E50915096C
:101B4D0070021508E4F508F5097D08FF1210A77D50
:101B5D00097F011210A77D0A7F021210A77D0B7F4E
:101B6D00031210A7E4FF1225187F011225187F021A
:101B7D001225187F0312251812281EEF7003021A62
:101B8D006D900261E0FFB40B02D212EF6431703A36
:101B9D0090025EE0FF900262E06F702E1229D3502A
:101BAD00FB90025EE0FF122DA8900263E0FFA3E020
:101BBD00FDA3E0FBA3E090022EF01217E01229D353
:101BCD0050FB90025EE0FF122D93900261E06432B3
:101BDD00703490025EE0FF900262E06F702812296F
:101BED00D350FB90025EE0FF122DA8900263E0FF40
:101BFD00A3E0FDA3E0FB121EBB1229D350FB900204
:101C0D005EE0FF122D93900261E0642D7039900219
:101C1D005EE0FF900262E06F702D1229D350FB90B1
:101C2D00025EE0FF122DA81229D350FB900263E053
:101C3D00FFA3E0FDA3E0FB1221201229D350FB905E
:101C4D00025EE0FF122D93900261E0642E703990D8
:101C5D00025EE0FF900262E06F702D1229D350FBFF
:101C6D0090025EE0FF122DA81229D350FB90026363
:101C7D00E0FFA3E0FDA3E0FB1221F01229D350FBFE
:101C8D0090025EE0FF122D93301352900261E0FF3F
:101C9D0020E726146016047044900262E090026CF6
:101CAD00F0122912122E2F122DBD8031900262E0FA
:101CBD0090026CF0122E80802490022AE0FEC00665
:101CCD00782B7C027D017B017A0279607E007F0793
:101CDD0012155F1225ECD0E04F90022AF0900261B0
:101CED00E0FFB41406D213C219C2A5EF6415600348
:0A1CFD00021A6DC213D2A5122E22A6
:031D0700021A6D50
:1022B500E5B0541EF52430A403432401E524653814
:1022C500600CE5246538F526753103852438E5313C
:1022D50060501531E531704AE52630E108E52420E6
:1022E500E103752502E52630E208E52420E20375C1
:1022F5002504E52630E308E52420E303752508E5F4
:102305002630E408E52420E403752510E52630E0B1
:1023150011E52420E00C90025C740FF0A374A0F08A
:10232500D21430143190025DE024FFF090025CE09D
:1023350034FFF0E5A030E405752501C21490025C78
:10234500E07002A3E0700FC21430120A90025EE042
:10235500FF7D06122996E51345126011E513151345
:0E236500700215121445127004C2A6C2A722FF
:032E9200D2FA224F
:1029EE008533A390025974FFF0A3742EF0A3749252
:0229FE00F022C5
:102D6500C2FAE5324528F5A390025974FFF0A37421
:072D750029F0A374EEF02227
:031A15000226E1C5
:1026E100C0E0C0F0C083C082C0D075D000C000C0BF
:1026F10001C002C003C004C005C006C007C2FF90EC
:102701000259A3E0FAA3E0F91217DAD007D006D0F4
:1027110005D004D003D002D001D000D0D0D082D0D7
:0627210083D0F0D0E0328D
:031A120002258426
:10258400C0E0C083C082C0D075D000C000C006C007
:1025940007C2CFE52725E02429F8E6FE08E625E072
:1025A400FFEE33FE74A72FF58274083EF583E4939F
:1025B400F532740193F533E527902E7593F52805CC
:1025C40027E527B4040375270090025974FFF0A38C
:1025D400742DF0A37465F0D2FFD007D006D000D0DC
:0825E400D0D082D083D0E03298
:031A2D0002276D20
:10276D00C0E0C0F0C083C082C0D075D000C000C032
:10277D0001C002C003C004C005C006C00753917F4D
:10278D001222B575E89075BB01D007D006D005D0E3
:10279D0004D003D002D001D000D0D0D082D083D0CD
:0427AD00F0D0E03256
:031A21000227B1E8
:1027B100C0E0C0D075D000C000C007C2EDE5BB606D
:1027C10019AFBB74132FF8A6BE75E890E5BBB40B27
:1027D1000575BB00800905BB800585BE1FD211D0E0
:0827E10007D000D0D0D0E03297
:1008A7000000000000000000000000040004000435
:1008B700000400040004000400040004000400080D
:1008C70000080008000800080008000800080008E1
:1008D7000008000C000C000C000C000C000C000CB5
:1008E700000C000C000C001000100010001000108D
:1008F7000010001000100010001000140014001465
:10090700001400140014001400140014001400183C
:100917000018001800180018001800180018001810
:100927000018001C001C001C001C001C001C001CE4
:10093700001C001C001C00200020002000200020BC
:100947000020002000200020002000240024002494
:10095700002400240024002400240024002400286C
:100967000028002800280028002800280028002840
:100977000028002C002C002C002C002C002C002C14
:10098700002C002C002C00300030003000300030EC
:1009970000300030003000300030003400340034C4
:1009A700003400340034003400340034003400389C
:1009B7000038003800380038003800380038003870
:1009C7000038003C003C003C003C003C003C003C44
:1009D700003C003C003C004000400040004000401C
:1009E70000400040004000400040004400440044F4
:1009F70000440044004400440044004400440048CC
:100A0700004800480048004800480048004800489F
:100A17000048004C004C004C004C004C004C004C73
:100A2700004C004C004C005000500050005000504B
:100A37000050005000500050005000540054005423
:100A470000540054005400540054005400540058FB
:100A570000580058005800580058005800580058CF
:100A67000058005C005C005C005C005C005C005CA3
:100A7700005C005C005C006000600060006000607B
:100A87000060006000600060006000640064006453
:100A9700006400640064006400640064006400682B
:100AA70000680068006800680068006800680068FF
:100AB7000068006C006C006C006C006C006C006CD3
:100AC700006C006C006C00700070007000700070AB
:100AD7000070007000700070007000740074007483
:100AE700007400740074007400740074007400785B
:100AF700007800780078007800780078007800782F
:100B07000078007C007C007C007C007C007C007C02
:100B1700007C007C007C00800080008000800080DA
:100B270000800080008000800084008400840084AE
:100B37000084008400840084008400840088008886
:100B4700008800880088008800880088008800885E
:100B5700008C008C008C008C008C008C008C008C2E
:100B6700008C009000900090009000900090009002
:100B770000900090009000940094009400940094DA
:100B870000940094009400940098009800980098AE
:100B9700009800980098009800980098009C009C86
:100BA700009C009C009C009C009C009C009C00A05A
:100BB70000A000A000A000A000A000A000A000A02E
:100BC70000A400A400A400A400A400A400A400A4FE
:100BD70000A400A800A800A800A800A800A800A8D2
:100BE70000A800A800AC00AC00AC00AC00AC00ACA6
:100BF70000AC00AC00B000B000B000B000B000B076
:100C070000B000B000B000B400B400B400B400B449
:100C170000B400B400B400B800B800B800B800B819
:100C270000B800B800B800BC00BC00BC00BC00BCE9
:100C370000BC00BC00BC00C000C000C000C000C0B9
:100C470000C000C000C000C400C400C400C400C489
:100C570000C400C400C800C800C800C800C800C855
:100C670000C800CC00CC00CC00CC00CC00CC00CC21
:100C770000D000D000D000D000D000D000D000D4E9
:100C870000D400D400D400D400D400D400D800D8B5
:100C970000D800D800D800D800DC00DC00DC00DC7D
:100CA70000DC00DC00E000E000E000E000E000E045
:100CB70000E400E400E400E400E400E400E800E805
:100CC70000E800E800E800E800EC00EC00EC00ECCD
:100CD70000EC00F000F000F000F000F000F400F489
:100CE70000F400F400F400F400F800F800F800F84D
:100CF70000FC00FC00FC00FC00FC010001000100FE
:100D070001000100010401040104010401080108B4
:100D1700010801080108010C010C010C010C01106C
:100D2700011001100110011401140114011401181C
:100D3700011801180118011C011C011C011C0120CC
:100D47000120012001240124012401240128012874
:100D57000128012C012C012C012C0130013001301C
:100D6700013401340134013801380138013C013CB8
:100D7700013C013C0140014001400144014401485C
:100D870001480148014C014C014C015001500150F0
:100D970001540154015801580158015C015C015C80
:100DA7000160016001640164016401680168016C0C
:100DB700016C017001700170017401740178017890
:100DC700017C017C0180018001800184018401880C
:100DD7000188018C018C0190019001940194019884
:100DE7000198019C019C01A001A401A401A801A8EC
:100DF70001AC01AC01B001B001B401B801B801BC4C
:100E070001BC01C001C401C401C801C801CC01D0A3
:100E170001D001D401D801D801DC01DC01E001E4F3
:100E270001E801E801EC01F001F001F401F801F833
:100E370001FC0200020402040208020C0210021064
:100E470002140218021C0220022002240228022C8B
:100E57000230023002340238023C024002440248A7
:100E6700024C024C025002540258025C02600264B7
:100E77000268026C027002740278027C02800284AB
:100E87000288028C029002940298029C02A002A49B
:100E970002A802AC02B002B802BC02C002C402C877
:100EA70002CC02D002D802DC02E002E402EC02F03B
:100EB70002F402F802FC03040308030C03140318EA
:100EC700031C03240328032C03340338034003447F
:100ED700034803500354035C03600368036C037403
:100EE700037803800384038C03900398039C03A473
:100EF70003AC03B003B803C003C403CC03D403D8C3
:100F070003E003E803F003F403FC0404040C0414F3
:100F1700041804200428043004380440044804500A
:100F270004580460046804700478048004880490FA
:100F3700049804A004A804B004B804C404CC04D4DE
:100F470004DC04E804F004F80500050C0514051C8E
:100F570005280530053C0544054C05580560056C1A
:100F670005740580058C059405A005A805B405C082
:100F770005C805D405E005EC05F40600060C0618BF
:100F870006240630063806440650065C06680674D2
:100F97000680068C069806A806B406C006CC06D8B6
:100FA70006E406F40700070C071C07280734074464
:100FB70007500760076C077C0788079807A407B4E2
:100FC70007C407D007E007F007FC080C081C082C2B
:100FD700083C084C085C086808780888089C08AC36
:100FE70008BC08CC08DC08EC08FC0910092009300B
:100FF70009440954096409780988099C09AC09C09E
:1010070009D409E409F80A0C0A1C0A300A440A58E8
:101017000A6C0A800A940AA80ABC0AD00AE40AF8E9
:101027000B0C0B200B340B4C0B600B740B8C0BA0B5
:101037000BB80BCC0BE40BF80C100C280C3C0C5425
:101047000C6C0C840C9C0CB40CCC0CE40CFC0D1438
:101057000D2C0D440D5C0D780D900DA80DC40DDC05
:101067000DF80E100E2C0E440E600E7C0E940EB072
:101077000ECC0EE80F040F200F3C0F580F740F9083
:101087000FB00FCC0FE80FFC0FFC0FFC0FFC0FFC91
:101097000FFC0FFC0FFC0FFC0FFC0FFC0FFC0FFCF1
:0F25EC0090022CE0FF540FFEEF54F06490703B10
:1025FB0090022EE0900232F090025EE06448702868
:10260B00EE30E306900232E0F534EE30E206900253
:10261B0032E0F535EE30E106900232E0F536EE3081
:0B262B00E006900232E0F5377F00224D
:10263600EF54F0FFBF800990025EE0B44802AF0697
:012646002271
:042E630041026D04B7
:10248E0090022B7403F0E4A3F0FFA3F0121A247E43
:10249E002A7F007B017A02792B900233E4F0A304A9
:1024AE00F0122727E4FF74492FF8E4F60FEFB40477
:1024BE00F5E4F545F546F547F54890022CF0900207
:1024CE002CE0FFC39463502A75F008EFA42401F5A5
:1024DE0082E5F0342AAF82FE7B007A0079459002C5
:1024EE0033E4F0A37408F012272790022CE004F0D6
:1024FE0080CC7E2D7F197B017A02792D900233E4F8
:0A250E00F0A304F01227270228A30F
:1029340090026DE0600414F0800B2012082015054D
:10294400D21553A0DF201906301303122E6AD219B0
:012954002260
:102D3400902D19E493600C902A00E49364036003DB
:092D440012248EE490026CF022CE
:1029120090026CE075F008A42401F9742A35F0FAEB
:102922007BFF78457C007D007E007F0812155FC228
:02293200192268
:10284E00121A2490026CE075F008A42401F582E5BA
:10285E00F0342AAF82FE7B007A007945900233E491
:0B286E00F0A37408F01227270228A333
:062E800012284EC21922C7
:0A17E00090022CEDF090022BEFF0C8
:1017EA00D39B50030218C0E024FFFEE434FF9002AA
:1017FA0030F0A3CEF0EB1490022FF090022CE024EC
:10180A00FFFFE434FFFE900230E0FCA3E0FDD39F2B
:10181A00EE6480F8EC6480984003021993EDAE04FC
:10182A007803C333CE33CED8F92401F582742A3E25
:10183A00AF82900237F0A3EFF090022FE075F00824
:10184A00A42401F9742A35F0FA90023474FFF0A343
:10185A00EAF0A3E9F0E4900232F0A3F0900234A394
:10186A00E475F0011215D8FEAFF0900237E475F076
:10187A00011215D885F082F583E493FD1223739043
:10188A000233E004F07006900232E004F0C39002E2
:10189A0033E09408900232E0940040C01228A390EA
:1018AA000231E004F07006900230E004F090022F5A
:1018BA00E004F002180590022CE024FFFEE434FF55
:1018CA00900230F0A3CEF090022EE014A3F0900222
:1018DA002BE024FFFFE434FFFE900230E0FCA3E09B
:1018EA00FDC39FEE6480F8EC64809850030219935C
:1018FA00EDAE047803C333CE33CED8F92401F58292
:10190A00742A3EAF82900237F0A3EFF090022FE0E4
:10191A0075F008A42401F9742A35F0FA9002347497
:10192A00FFF0A3EAF0A3E9F0E4900232F0A3F0900A
:10193A000234A3E475F0011215D8FEAFF090023715
:10194A00E475F0011215D885F082F583E493FD124F
:10195A002373900233E004F07006900232E004F040
:10196A00C3900233E09408900232E0940040C0121F
:10197A0028A3900231E024FFF0900230E034FFF017
:09198A0090022FE014F00218D8BD
:011993002231
:051EBB0090022BEDF088
:101EC000EF14900239F0EB14A3F090022BE014FF12
:101ED000900239E0D39F400302201AA3E075F00876
:101EE000A42401F582E5F0342AAF82FEE490023B9F
:101EF000F0A3F090023BE0FCA3E0FDC39408EC9457
:101F000000502B0FEFAA0670010E14F5828A83E4AD
:101F100093FB74312DF582E43402F583EBF09002EB
:101F20003CE004F070CD90023BE004F080C59002EC
:101F30003AE075F008A42401F9742A35F0FA900209
:101F40002C74FFF0A3EAF0A3E9F0900239E075F0F9
:101F500008A42401F582E5F0342AAF8290022FF024
:101F6000A3EFF0E490023BF0A3F090022CA3E47501
:101F7000F0011215D8FEAFF090022FE475F00112B7
:101F800015D885F082F583E493FD12237390023C0B
:101F9000E004F0700690023BE004F0C390023CE0E5
:101FA000940890023BE0940040C0900239E075F044
:101FB00008A42401F9742A35F0FA90022C74FFF079
:101FC000A3EAF0A3E9F0E490023BF0A3F090023B17
:101FD000E0FCA3E0FDC39408EC9400502D90022C8B
:101FE000A3E475F0011215D8FEAFF074312DF5821F
:101FF000E43402F583E0FD12237390023CE004F028
:1020000070CB90023BE004F080C31228A390023909
:0A201000E004F0A3E004F0021ECA91
:01201A0022A3
:0721F00090022BEBF0AC079D
:1021F700A3E5C1F0A2AFE433A3F0AF05A3E4F0A3D6
:10220700EFF0E07F00FE90022EF0A3EFF0AD04EDBB
:10221700FF90022EEEF0A3EFF0C2AF43C15D900234
:102227006C740FF0121A2490026CE075F008A42465
:1022370001F9742A35F0FA90023074FFF0A3EAF03E
:10224700A3E9F0E4A3F090022EE0FCA3E0FFECFD8D
:1022570090022BE0FBE4900238F0D20912201B9089
:102267000234EFF0FD900230A3E475F0011215D8A7
:10227700FEAFF012237390022FE004F07006900275
:102287002EE004F0900233E004F0E0C3940840B677
:102297001228A390026CE004F0E0C3941E408590DE
:0E22A700022CE0F5C1A3E024FF92AF022E79D5
:0721200090022BEBF0AC076D
:10212700A3E5C1F0A2AFE433A3F0AF05900230E41A
:10213700F0A3EFF0E07F00FE900230F0A3EFF0ADE8
:1021470004EDFF900230EEF0A3EFF0C2AF43C15DA4
:1021570090026C740FF090026CE0FFC3941E507AEB
:1021670075F008EFA42401F582E5F0342AAF8290D8
:102177000232F0A3EFF0E490022EF0A3F0900230C9
:10218700E0FCA3E0FFECFD90022BE0FB900232E4C1
:1021970075F0011215D885F082F583E49390023823
:1021A700F0C20912201B900231E004F07006900281
:1021B70030E004F090022FE004F0700690022EE069
:1021C70004F0C390022FE0940890022EE0940040A0
:1021D700AC90026CE004F002215D90022CE0F5C1A6
:0921E700A3E024FF92AF022E795F
:0528EE0090024CEDF02A
:1028F30090024D74FF121744EC4D4E4F601090023E
:0E2903004CE012159E740129F9E43AFA80E2C4
:0129110022A3
:102D7C00E4FD0FEFAA0670010E14F5828A83E06061
:062D8C00030D80EEAF050F
:012D9200221E
:10264700900251EBF0A3EAF0A3E9F090025774FF70
:10265700F5F01215D845F06034900254E0FBA3E082
:10266700FAA3E0F9121585FF900251E0FBA3E0FA07
:10267700A3E0F9EF12159E900252E475F0011215CE
:0E268700C2900255E475F0011215C280BE2209
:10297600A2AFE433FDC2AF758F0375B7A575B7F186
:0F2986008F828E83E4F0F58FAF05EF24FF92AFC1
:01299500221F
:10295500A2AFE433FCC2AF758F0175B7A575B7F1AA
:102965008F828E83EDF0E4F58FAF04EF24FF92AFF5
:01297500223F
:10269500900243EEF0A3EFF0A3ECF0A3EDF0EB4ACC
:1026A5006039900243E0FEA3E0FFA3E0FCA3E0F560
:1026B500828C83E0FD122955EB1B70011A900246AE
:1026C500E004F07006900245E004F0900244E00456
:0C26D500F070CB900243E004F080C322C0
:081A2400E4900000F0A3F022A1
:1028A300900000E0FEA3E0FF122976900000E0FE16
:1028B300A3E0FF7C007D027B007A02122695E49060
:0628C3000000F0A3F0226A
:0A237300A90590023DEEF0A3EFF083
:10237D00EE54FEFE900000E0FCA3E0FD7002EE6C5A
:10238D006059ED4C60031228A390023DE0FEEE541F
:10239D00FEFE7F00900000F0A3EFF090023FEEF004
:1023AD00A3EFF0A37400F0A37402F07F007E0290FF
:1023BD00023FE475F0011215D885F082F583E493A0
:1023CD00FD900241E475F0011215D885F082F58378
:1023DD00EDF0EF1F70011EEF4E70D490023DE0FC4A
:1023ED00A3E0FDEC5401FC74022DF58274003CF564
:0323FD0083E9F081
:0124000022B9
:1027270090022EEEF0A3EFF0A3EBF0A3EAF0A3E9FB
:10273700F090023374FFF5F01215D845F06026903B
:10274700022EE475F0011215D8AFF0FE900230E0CA
:10275700FBA3E475F0011215D8A9F0FA121585FD4F
:0627670012237380CC2256
:10299600900247EFF0A3EDF07F0A12240190024760
:1029A600E0FF122401900248E0FF122401022E7972
:082E6A007F02122401022E79FF
:06281E00122E86EF602778
:1028240090022B7402F0A37460F012287990022BAA
:10283400E475F0011215D885F082F583EFF0122EBD
:072844008CEF70E67F01221A
:03284B007F0022E9
:102D930090022BEFF07F2F12240190022BE0FF1201
:052DA3002401022E795D
:102DA80090022BEFF07F3012240190022BE0FF12EB
:052DB8002401022E7948
:022E6700C11791
:1029D300E53CB54014E53BB53F0FE53CB5440AE59E
:0B29E3003BB5430520C502D322C322F0
:0C2E4800758920438E08758DE8D28E221B
:102DF70075C101E4F5C2F5C053C17F43C180022EFE
:012E07004882
:1028C9007E027F028E3D8F3E8E418F428E398F3A36
:1028D9007E027F168E3F8F408E438F448E3B8F3C06
:0528E900C216022DF7EC
:1027E9000542E542AA417002054114F5828A83EF48
:1027F900F0AF050542E542AC417002054114F5828E
:102809008C83EFF07416B5420B7402B5410675411D
:052819000275420222DD
:072E7900C216C2C4D2C5223B
:10240100201645D2160544E544AC43700205431439
:10241100F5828C8374FFF07C027D2AEDB5440AECD1
:10242100B543067543027544160544E544AA437055
:1024310002054314F5828A83E4F0EDB5440AECB554
:1024410043067543027544160544E544AC437002E6
:10245100054314F5828C83E4F07C027D2AEDB544BA
:102461000AECB543067543027544160544E544AAD2
:10247100437002054314F5828A83EFF0EDB5440AF7
:0D248100ECB543067543027544167F012239
:1029B600E53AB53E08E539B53D037F0022853E82FE
:0D29C600853D83E0B507037F01227F0022DD
:10287900053EE53E7002053D053EE53EAE3D700272
:10288900053D14F5828E83E0FF7416B53E0B740284
:09289900B53D06753D02753E02D5
:0128A2002213
:062E86007FFF1229B622B5
:062E8C00E4FF1229B6224A
:031A1800021D0AA2
:101D0A00C0E0C083C082C0D075D000C000C002C08D
:101D1A0004C005C006C007E5C054FE1217B41E82EF
:101D2A00081E820A1E980C1E980E1E61101E611251
:101D3A001E74141E74161E591C1E591E1E55241E6E
:101D4A0055261E16281E162A1E242C1E242E1DA4B5
:101D5A00C01DB1C21D68E01D68E200001EA4C2C514
:101D6A00053CE53C7002053B7E027F2AB5070AEE78
:101D7A00B53B06753B02753C16053CE53CAC3B7031
:101D8A0002053B14F5828C83E0F5C2EF653C7003D3
:101D9A00EE653B6003021EA48069853F3B85403C9B
:101DAA00D2C4D2C5021EA4E53CB54412E53BB543F4
:101DBA000D85433F854440C2C5D2C4021EA4853C5A
:101DCA0082853B83E0B4FF03021EA0053CE53C701C
:101DDA0002053B7E027F2AB5070AEEB53B06753B34
:101DEA0002753C16053CE53CAC3B7002053B14F51C
:101DFA00828C83E0F5C2EF653C7003EE653B6003BD
:101E0A00021EA4753B02753C16021EA4E5C2602A96
:101E1A0090025EE065C260228016853F3B85403CA9
:101E2A00C2C5D217E5C2601290025EE065C2600ABE
:101E3A00C2C4C2C5C2C1C2188060ADC27FFF122728
:101E4A00E9C2C4C2C5D2C1D218804FD2C5804B855F
:101E5A003B3F853C40804385413985423AC2C4C2F2
:101E6A00C1301736D2C5C2178030853F3B85403C0A
:101E7A00C2C4C2C1D2C58022C2C4C2C5201804C20B
:101E8A00C18017ADC2E4FF1227E9D2C1800C853F99
:101E9A003B85403CC2C1C2C4D2C5C2C0D007D0062D
:101EAA00D005D004D002D000D0D0D082D083D0E0E8
:011EBA0032F5
:0D2E2200D204D203D202D201C2A6C2A7225E
:0D2E2F00C204C203C202C201C2A6C2A72291
:0710A70090022BEFF0AB05F6
:1010AE00C2AFC200E0FF240AF8E690026BF0FD74B6
:1010BE00142BF8E6F9C39DFCE4940090022CF0A3E7
:1010CE00CCF030054D90022CE0FCA3E0FDC3EC64A7
:1010DE00809480502E740E2FF8E6700276039002E4
:1010EE002BE0FF240EF816E66003021183740E2F18
:1010FE00F8760174142BF8E6FE740A2FF8A606D2C1
:10110E00008072D3ED9404EC64809480405EC2053E
:10111E00804D90022CE0FEA3E0FFD39400EE64809D
:10112E009480402E90022BE0240EF8E67002760397
:10113E0090022BE0FD240EF816E67039740E2DF891
:10114E00760174142BF8E6FC740A2DF8A604D2006E
:10115E008023C3EF94FCEE6480947F500FD20590F1
:10116E00022BE0240AF8A601D200800990022BE09F
:10117E00240EF8E4F6E5094508600302148C2000FD
:10118E000302148C90022BE0FD2449F8E6FE7467EE
:10119E002DF582E43402F583E0FDEDFFE4FCFD90D5
:1011AE00022E12177790022CE0FEA3E0FFD39400DC
:1011BE00EE6480948050030212CFEE3395E0FDFC76
:1011CE00781012172F900232121777900232E0FC2D
:1011DE00A3E0FDA3E0FEA3E0FFC006C00790026BF4
:1011EE00E0FFC374FF9FFFE49400AB07FAE4F9F845
:1011FE00D007D0061216799002321217779002326B
:10120E00E0F8A3E0F9A3E0FAA3E0FBC00090022B04
:10121E00E02449F8E6FFC374FF9FFFE49400FEE468
:10122E00FCFDD0001215EE90023212177790022BB1
:10123E00E02449F8E6FF90026BE0D39F900232E083
:10124E00FCA3E0FDA3E0FEA3E0FFE440067B407AB2
:10125E000180037BC0FAF9F81215EE9002321217D4
:10126E007790022EE0F8A3E0F9A3E0FAA3E0FBC02A
:10127E0000A3E0FCA3E0FDA3E0FEA3E0FF781012C4
:10128E00171CD000EB2FFFEA3EFEE93DFDE83CFCCB
:10129E0090022E121777E47FFF7EFFFDFC90022E48
:1012AE00E0F8A3E0F9A3E0FAA3E0FBD312170B508A
:1012BE00030213DD90022E1217830000FFFF0213AC
:1012CE00DD90022CE0FEA3E0FFC3E49FFFE49EFE50
:1012DE003395E0FDFC781012172F9002321217771B
:1012EE00900232E0FCA3E0FDA3E0FEA3E0FFC00706
:1012FE0090026BE0FBE4FAF9F8D00712167990022F
:10130E0032121777900232E0F8A3E0F9A3E0FAA3C5
:10131E00E0FBC00090022BE02449F8E6FFE4FCFD60
:10132E00FED0001215EE90023212177790022BE0CB
:10133E002449F8E6FF90026BE0C39F900232E0FC76
:10134E00A3E0FDA3E0FEA3E0FFE450067B407A019C
:10135E0080037BC0FAF9F81215EE9002321217775D
:10136E0090022EE0FCA3E0FDA3E0FEA3E0FFC0048C
:10137E00C005C006C007A3E0FCA3E0FDA3E0FEA3EA
:10138E00E0FF781012171CA804A905AA06AB07D017
:10139E0007D006D005D004C3EF9BFFEE9AFEED9961
:1013AE00FDEC98FC90022E121777E47FFF7EFFFD76
:1013BE00FC90022EE0F8A3E0F9A3E0FAA3E0FBD341
:1013CE0012170B400A90022E121783000000009095
:1013DE00022EA3A3A3E0FF90022BE0FB2467F5826D
:1013EE00E43402F583EFF090022EE0FCA3E0FDA3BF
:1013FE00E0FEA3E0FF780812171C90022E1217775A
:10140E0074492BF8E6FFE4FCFDFE90022EE0F8A3F3
:10141E00E0F9A3E0FAA3E0FBC312170B60149002ED
:10142E002EA3A3A3E0FF90022BE02449F8A60712F7
:10143E00293430052890022BE0FF240AF8E6FE241A
:10144E0004FDE433FC74492FF8E6FFD39DEC648071
:10145E00F87480985028EFC39E4023801D90022B75
:10146E00E0FF240AF8E6FE74492FF8E6FFD39E50FB
:10147E000DEE24FCFEEFC39E4004C2A6C2A7D2AF5F
:01148E00223B
:03000000020800F3
:03000300021A03DB
:03000B00021A06D0
:03001300021A09C5
:03001B00021A0CBA
:03002300021A0FAF
:03002B00021A12A4
:03003300021A1599
:03003B00021A188E
:03004300021A1B83
:03004B00021A1E78
:03005300021A216D
:03005B00021A2462
:03006300021A2757
:03006B00021A2A4C
:03007300021A2D41
:10080000E4F5D9E5EF7480F5FF7402F5EF787FE445
:10081000F6D8FD9000007F007E04E4F0A3DFFCDE4C
:07082000FA75814C02086229
:08201B00900235EFF0A3EDF097
:10202300A209920DC20F201BFDD21B900239EBF0C7
:10203300C20AD20BD20E7F01C2C4C210D2C530C0B5
:10204300FDE5C054F0248070030220D524C0601B3A
:1020530024E06003022105900239E0F5C2A20AE4FC
:102063003342C2C2C5E4A3F002210730C159301084
:1020730007D2C5C210022107300B0CC20BD20C9041
:102083000236E0F5C2807D300C11C20C900235E0BF
:10209300F5C2300D6FD210D20A8069200A66EFFDB7
:1020A30090023AE0FB3395E0FAC3EB9D7480F86A43
:1020B30098500E900238E0F5C290023AE004F080A6
:1020C30043D2C4C21B803D300E04D2C58036D20F2A
:1020D3008032EFFD90023AE0FB3395E0FAC3EB9DCB
:1020E3007480F86A98500CA3E5C2F090023AE004B9
:1020F300F0D2C190023AE0B5070AC21BC2C1D2C4F2
:102103008002D20F300F0853C0BF43C040C21BC26E
:0C211300C0301B0302204190023BE0FFA3
:01211F00229D
:10082700021A30E493A3F8E493A34003F68001F29D
:1008370008DFF48029E493A3F85407240CC8C333D2
:10084700C4540F4420C8834004F456800146F6DFA1
:10085700E4800B0102040810204080902E5FE47EA4
:10086700019360BCA3FF543F30E509541FFEE49396
:10087700A360010ECF54C025E060A840B8E493A35D
:10088700FAE493A3F8E493A3C8C582C8CAC583CA88
:10089700F0A3C8C582C8CAC583CADFE9DEE780BE40
:012E69000068
:10148F00E709F608DFFA8046E709F208DFFA803E3F
:10149F0088828C83E709F0A3DFFA8032E309F6082C
:1014AF00DFFA8078E309F208DFFA807088828C8394
:1014BF00E309F0A3DFFA806489828A83E0A3F60848
:1014CF00DFFA805889828A83E0A3F208DFFA804C22
:1014DF0080D280FA80C680D4806980F280338010F9
:1014EF0080A680EA809A80A880DA80E280CA803362
:1014FF0089828A83ECFAE493A3C8C582C8CCC583DA
:10150F00CCF0A3C8C582C8CCC583CCDFE9DEE780A9
:10151F000D89828A83E493A3F608DFF9ECFAA9F028
:10152F00EDFB2289828A83ECFAE0A3C8C582C8CC7E
:10153F00C583CCF0A3C8C582C8CCC583CCDFEADE97
:10154F00E880DB89828A83E493A3F208DFF980CCF9
:10155F0088F0EF60010E4E60C388F0ED2402B404F2
:10156F000050B9F582EB2402B4040050AF23234599
:06157F0082239014DF73CB
:10158500BB010689828A83E0225002E722BBFE0264
:09159500E32289828A83E4932297
:10159E00BB010689828A83F0225002F722BBFE012C
:0215AE00F32226
:1015B000EF8DF0A4A8F0CF8CF0A428CE8DF0A42E4F
:0215C000FE2209
:1015C200C5F0F8A3E028F0C5F0F8E58215827002B4
:0615D2001583E038F02251
:1015D800A3F8E0C5F025F0F0E582158270021583C6
:0615E800E0C838F0E82223
:1015EE00E88FF0A4CC8BF0A42CFCE98EF0A42CFC9C
:1015FE008AF0EDA42CFCEA8EF0A4CDA8F08BF0A41A
:10160E002DCC3825F0FDE98FF0A42CCD35F0FCEB78
:10161E008EF0A4FEA9F0EB8FF0A4CFC5F02ECD393D
:0F162E00FEE43CFCEAA42DCE35F0FDE43CFC22AA
:10163D0075F008758200EF2FFFEE33FECD33CDCC64
:10164D0033CCC58233C5829BED9AEC99E5829840E7
:10165D000CF582EE9BFEED9AFDEC99FC0FD5F0D6C4
:10166D00E4CEFBE4CDFAE4CCF9A88222B800C1B9EE
:10167D000059BA002DEC8BF084CFCECDFCE5F0CB2C
:10168D00F97818EF2FFFEE33FEED33FDEC33FCEB65
:10169D0033FB10D703994004EB99FB0FD8E5E4F920
:1016AD00FA227818EF2FFFEE33FEED33FDEC33FC0D
:1016BD00C933C910D7059BE99A4007EC9BFCE99A01
:1016CD00F90FD8E0E4C9FAE4CCFB2275F010EF2F46
:1016DD00FFEE33FEED33FDCC33CCC833C810D70746
:1016ED009BEC9AE899400AED9BFDEC9AFCE899F881
:0E16FD000FD5F0DAE4CDFBE4CCFAE4C8F92214
:10170B00EB9FF5F0EA9E42F0E99D42F0E89C45F034
:01171B0022AB
:10171C00E8600FECC313FCED13FDEE13FEEF13FFAB
:03172C00D8F122CF
:10172F00E8600FEFC333FFEE33FEED33FDEC33FC18
:03173F00D8F122BC
:101742007401FF3395E0FEFDFCA3A3A3E0CF2FF0CD
:10175200E582158270021583E0CE3EF0E5821582A5
:1017620070021583E0CD3DF0E5821582700215838B
:05177200E0CC3CF02278
:0C177700ECF0A3EDF0A3EEF0A3EFF022E5
:10178300A8828583F0D083D08212179A12179A12F7
:10179300179A12179AE473E493A3C583C5F0C5831C
:1017A300C8C582C8F0A3C583C5F0C583C8C582C8B0
:0117B3002213
:1017B400D083D082F8E4937012740193700DA3A3C4
:1017C40093F8740193F5828883E4737402936860D8
:0617D400EFA3A3A380DFD8
:0617DA008A838982E4739A
:00000001FF
